:100000000C94A9050C94C6050C94C6050C94C60561
:100010000C94C6050C94C6050C94C6050C94C60534
:100020000C94C6050C94C6050C94FB090C94C605EB
:100030000C94C6050C94C6050C94C6050C94C60514
:100040000C94C6050C94EF060C948A2B0C945D2B33
:100050000C94C6050C94C6050C94C6050C94C605F4
:100060000C94C6050C94C6050C94C6050C94C605E4
:100070000C94C6050C94C6050C94C6050C94C605D4
:100080000C94C6050C94C6050C94C605456173799D
:10009000436F6E74726F6C00204C4300205043001D
:1000A000696E636F6D70617469626C65204857009A
:1000B000312E342E360001020317180405061511DF
:1000C00007080916120A000B0C13100F0E0D140E60
:1000D000111116111116100A00111111110E001133
:1000E0000E111111110E0011040A11111F1100013E
:1000F0000101050D1F0C04040E1F04041F0E040053
:10010000060917170906000006091214120906034A
:10011000070F1E1C18100003050912141810000701
:100120000707070707070707050505050505070072
:1001300000001515171111171113111700000000F9
:1001400000001711171417121212121200000000EB
:10015000000017151515171C101815150701011C9F
:10016000101816110201061C101816110204071CA3
:1001700010181216020207040A110A0A0E00000CD7
:1001800017141714170C001C101810160505051F5E
:100190000A0A0A0A0A1F000E11111F1B1B1F000268
:1001A000060F1F0F060200080C1E1F1E0C08000E73
:1001B0000E0E0E1F0E0400040E1F0E0E0E0E00205B
:1001C0006D332020200000204D4D492020000020CC
:1001D0004D4D0120200000204443432020000020FA
:1001E00053544F5020000053484F525421000020D8
:1001F00048414C54200000202020202020000020D6
:1002000050524F47200000524553455420000020D3
:100210002054504D2000007E0E0E0E0E1B1B1C0E97
:100220001B1B7E0E0E0E0E253364002020202000A6
:10023000232D004144523A20256C642020202020A8
:100240002020202020002D2D2D2D202000252D3593
:10025000640025336400253364002020010220203F
:10026000202020202000252D356400252D31312E21
:10027000313173004142434445464748494A4B4C5B
:100280004D4E4F505152535455565758595A30317C
:1002900032333435363738392E2C3A2D2B232F3D37
:1002A0003C7C3E20004D4D20492020313420004D23
:1002B0004D20492020323761004D4D204920203209
:1002C0003762004D4D20012020313420004D4D205B
:1002D000012020323761004D4D200120203237624D
:1002E0000044434320202031342000444343202055
:1002F0002032382000444343202031323820006D22
:100300003320202031323820004C6F636F6D6F74C2
:10031000697665206D656E7500444343204D6169C3
:100320006E20547261636B00004443432052616944
:100330006C436F6D204356000053657474696E679B
:100340007300000000000000004C43442062616321
:100350006B6C696768740000004C6F6B436F6E7460
:10036000726F6C00000000000045786974000000A6
:1003700000000000000000000053656C65637420FD
:100380000000000000000000004461746120666FFE
:10039000726D617400000000004E616D65202020C8
:1003A000202020000000000000456E74727920209B
:1003B0002020200000000000003132384653204D3C
:1003C0006F64650000000000004A6F676469616C3B
:1003D000204D6F6465000000004C6F636D656E75A5
:1003E00000000000000000000044434320686F6FDD
:1003F000666473706F6F72000044434320526169FA
:100400006C436F6D2043560000496E7374656C6CCD
:10041000696E67656E000000004C4344207665728B
:100420006C69636874696E67004C6F6B436F6E74C0
:10043000726F6C00000000000045786974000000D5
:100440000000000000000000004B69657A656E2026
:1004500000000000000000000044617461666F72DB
:100460006D61740000000000004E61616D2020206D
:10047000202020000000000000496E766F65722089
:100480002020200000000000003132384653204D6B
:100490006F64650000000000004A6F676469616C6A
:1004A000204D6F6465000000004D656E75204C6F37
:1004B000636F0000000000000050726F6772616D92
:1004C0006D6174696F6E000000444343205261699E
:1004D0006C436F6D20435600005265676C61676521
:1004E0007300000000000000004C756D696E6F73B2
:1004F0006974650000000000004C6F6B436F6E7400
:10050000726F6C0000000000004578697400000004
:1005100000000000000000000053656C6563746912
:100520006F6E20000000000000466F726D61742045
:10053000646F6E6E65657300004E6F6D2020202025
:1005400020202000000000000053616973696520CD
:100550002020200000000000003132384653204D9A
:100560006F64650000000000004A6F676469616C99
:10057000204D6F6465000000004C6F6B204D656E70
:10058000FC00000000000000004443432048617567
:100590007074676C6569730000444343205261695D
:1005A0006C436F6D204356000045696E7374656C33
:1005B0006C756E67656E0000004C43442042656CAC
:1005C0006575636874756E67004C6F6B436F6E740E
:1005D000726F6C0000000000004578697400000034
:1005E00000000000000000000041757377E4686CB3
:1005F000656E20000000000000446174656E666F47
:10060000726D617400000000004E616D6520202055
:1006100020202000000000000045696E74726167B0
:100620002020200000000000003132384653204DC9
:100630006F64650000000000005265676C65726DB4
:100640006F6475730000000000202D2D2D2D0025F6
:10065000357500536F6674772E205600312E342E78
:1006600036005365724E722E2025386C75003A2084
:100670000025357500253364002534643A20002DAB
:100680002D2D0025336400204F4B202020200020FA
:1006900020202020202000202D2D2D002534640036
:1006A000696E636F6D7061742E20466F726D617438
:1006B00000496E636F6D702E20466F726D617420FD
:1006C0002000466F726D617420696E636F6D70619A
:1006D000742E00696E6B6F6D7061742E20466F72A0
:1006E0006D6174002E2E2E2077616974696E67200B
:1006F0002E2E2E2000233D64656C6574650000007D
:10070000000000000000286E6F20656E7472792969
:10071000000000000000002E2E2E2064656C657421
:10072000696E67202E2E2E00206661756C740000A5
:1007300000000000000000000020444343206F6ED2
:100740006C79212020202020200020707265737396
:1007500020474F20666972737400002A3D43616E22
:1007600063656C2020200000000000002070726F84
:100770006772616D696E670000000000002D73688C
:100780006F727420636972637569742D2000206E26
:1007900061746976652028313A31292020200020B3
:1007A0006C696E6561722028323A31292020200060
:1007B0002070726F677265737369766520312020CF
:1007C000002070726F6772657373697665203220DE
:1007D0002000204143204D6F6465202020202020F0
:1007E000202000204443204D6F64652020202020DD
:1007F000202020002E2E2E207761636874656E20E5
:100800002E2E2E2000233D77697373656E00000045
:10081000000000000000286765656E20696E766F35
:1008200065722900000000202E2E2E207769737338
:10083000656E202E2E2E000020666F75740000005D
:1008400000000000000000000020416C6C65656E37
:1008500020444343212020202000207072657373C0
:1008600020474F20666972737400002A3D2041665C
:100870006272656B656E0000000000002050726FB0
:100880006772616D6D6572656E000000002D2D4B05
:100890006F7274736C756974696E672D2D00206EAC
:1008A00061746976652028313A31292020200020A2
:1008B0006C696E6561722028323A3129202020004F
:1008C0002070726F677265737369766520312020BE
:1008D000002070726F6772657373697665203220CD
:1008E0002000204143204D6F6465202020202020DF
:1008F000202000204443204D6F64652020202020CC
:100900002020200050617469656E74657A000000D3
:100910000000000000233D7375707072696D657290
:10092000000000000000766964650000000000001F
:1009300000000000000000537570707265737369E9
:100940006F6E000000000000204572726575720035
:100950000000000000000000002044434320756EAA
:10096000697175656D656E742000207072657373B2
:1009700020474F20666972737400002A3D4162610E
:100980006E646F6E20200000000000002050726F27
:100990006772616D6D6174696F6E0000002D436F49
:1009A0007572742D636972637569742D2000206EF1
:1009B00061746976652028313A3129202020002091
:1009C0006C696E6561722028323A3129202020003E
:1009D0002070726F677265737369766520312020AD
:1009E000002070726F6772657373697665203220BC
:1009F0002000204143204D6F6465202020202020CE
:100A0000202000204443204D6F64652020202020BA
:100A1000202020002E2E2E2077617274656E202EED
:100A20002E2E202000233D4CF6736368656E000077
:100A3000000000000000286B65696E2045696E7437
:100A400072616729000000202E2E2E206CF6736341
:100A50006865202E2E2E2000204665686C65720089
:100A6000000000000000000000206E75722066FC8F
:100A7000722044434321202020002065727374209B
:100A8000474F206472FC636B656E002A203D204155
:100A90006262727563680000000000002050726F8F
:100AA0006772616D6D696572756E6700002D2D202E
:100AB0004B75727A7363686C75DF202D2D00204EA4
:100AC000617469762028313A3129202020200020C5
:100AD0004C696E6561722028323A3129202020004D
:100AE0002050726F67726573736976203120202001
:100AF000002050726F677265737369762032202010
:100B00002000204143204D6F647573202020202059
:100B1000202000204443204D6F6475732020202046
:100B2000202020005B6E6F206D6573736167655DCB
:100B3000005B756E6B6E6F776E206572726F725DA3
:100B4000004003A001CF00670044003300190010EB
:100B5000000011241FBECFEFD0E1DEBFCDBF11E0FA
:100B6000A0E0B1E0EAEEF5E600E00BBF02C00790BE
:100B70000D92A634B107D9F713E0A6E4B1E001C0A5
:100B80001D92A33BB107E1F70C940F060C940000F3
:100B900081E0809347010895482F9091460198176E
:100BA00031F0963021F0953029F4863019F080E04C
:100BB00090E0089540934601453021F460E280E0E2
:100BC0000E94232940914601463021F460E280E0F2
:100BD0000E942329809146010E94242D0E94C8056D
:100BE00081E090E008950895809146019927089545
:100BF00080E00E948D0E2FEF8F3F920721F0682F2B
:100C000080E00E94762D0E9485250E94DE1380914F
:100C10004701882311F40E943D0DA8950895CFEF58
:100C2000D0E1DEBFCDBF0E9402230E94AA0622E0CF
:100C30004EE468E083E00E941B2B0E94D00678946B
:100C40000E9479090E942823FC0184810E94A50D3D
:100C50006CE870E082E00E940B0E0E945A23823002
:100C600021F00E945A23813019F468E970E012C023
:100C70000E945A23803819F46CE970E00BC060E0E0
:100C800081E00E94530C60EA70E082E00E940B0E4B
:100C9000A895FECF82E00E940B0E60E081E00E94EA
:100CA000530C66E582E00E94AA0D60EB70E082E0E2
:100CB0000E940B0E0E942823EC0181E00E943E0B53
:100CC000882319F081E00E942B2382E00E943E0BD2
:100CD000882319F080E00E942B2383E00E943E0BC2
:100CE000882319F082E00E942B2384E00E943E0BAF
:100CF000882329F083E00E942B2301C0A8950E943D
:100D0000DE248823D9F360E070E089859A85009716
:100D100031F0AB010E94292ABC01892B11F46A81B0
:100D20007B818FEF0E94CA2381E011C00E942D14A5
:100D30000E94FF0BFFEF8F3F9F07C1F70E94F8054E
:100D4000809147018823A1F31092470180E00E941F
:100D50000311EECF8FE78ABB1BBA80E187BB18BABD
:100D600080EF84BB8FEF85BB8BEB81BB8CEC82BBB0
:100D700082E082B987EF83B987E78093610081EFD2
:100D8000809362008FE18093640089E18093650025
:100D90000E94B30AA89588E181BD8CE081BD0895C9
:100DA0000E944C239B01AC0193E0E92FFF27EE5AF0
:100DB000FE4F822F8F77808387E056954795379532
:100DC00027958A95D1F7915097FFEFCF87B3807F12
:100DD00087BB88B3807F88BB84EE8DB908951F924E
:100DE0000F920FB60F9211242F933F934F935F935F
:100DF0006F937F938F939F93EF93FF938091000165
:100E0000909101018F5F9F4F71F0BB9A809100011B
:100E10008FB9769B0BC0BB981092480110924F017E
:100E200010924E0103C0BB988FEF8FB97FB177FF4F
:100E30007FC08091500190915101892BE1F0809108
:100E40004C018F5F80934C0180914C01803210F0F7
:100E500010924C0190914C0180914D01981759F4DA
:100E600080914D018F5F80934D0180914D018032C3
:100E700010F010924D0180914E0190914F018A51D6
:100E8000934061F058F080914B018F5F80934B014C
:100E900080914B01843010F010924B01109251015F
:100EA0001092500110924F0110924E016091430137
:100EB000761721F481E08093480171C010924801B7
:100EC000472F55279A012F773070862F992728179B
:100ED000390721F07F3F11F06F3F61F490914C0191
:100EE00089E0989FC001112486509E4F9093510134
:100EF000809350014F775070862F992748175907D4
:100F000009F04DC090914A0180914B01981749F02A
:100F100090914B0189E0989FC0011124865E9C4FFF
:100F200002C081EF91E090934F0180934E0137C052
:100F300020914801822F99278130910531F081302D
:100F400091056CF106975CF516C02F5F2093480160
:100F5000703419F41092490122C0713411F481E007
:100F600007C0723411F482E003C0733491F483E05B
:100F70008093490114C0E22FFF27809149019927EE
:100F800002968E179F0744F0E05BFE4F8081781732
:100F900019F01092480103C02F5F209348018091FF
:100FA0004801882339F480914E0190914F01892B9B
:100FB00079F003C0872F99270DC0E0914E01F09181
:100FC0004F0181919927F0934F01E0934E0102C0A8
:100FD0008FEF9FEF9093010180930001809150016A
:100FE000909151018A51934020F01092510110923A
:100FF0005001E0915001F0915101309729F0719327
:10100000F0935101E0935001FF91EF919F918F91E7
:101010007F916F915F914F913F912F910F900FBEF4
:101020000F901F901895DC0180914A01282F3327DB
:1010300080914B01992701972817390741F080913A
:101040004A01833039F480914B01882319F480E000
:1010500090E0089590914A0189E0989FF001112451
:10106000E65EFC4F98E08D918193915097FFFBCF06
:1010700080914A018F5F80934A0180914A018430B8
:1010800010F010924A0181E090E008950895FC016B
:10109000A1EFB1E098E081918D93915097FFFBCF44
:1010A00008959C0190914C0180914D01981719F47D
:1010B00080E090E00895D9012115310511F4C901AE
:1010C0000895F89490914D0189E0989FF0011124C2
:1010D000E650FE4F98E081918D93915097FFFBCFA2
:1010E00080914D018F5F80934D0180914D01803241
:1010F00010F010924D017894C901089508950000F0
:101100000000000000000895882341F080916500F0
:101110008460809365000E947F0808958091650037
:101120008B7F80936500089508951F93182F8AB3CD
:10113000807F8ABB80E00E94840880916500826085
:1011400080936500112321F080916500816003C0C8
:10115000809165008E7F809365000000000081E033
:101160000E94840819B380E00E9484081295107FC1
:101170000E947F0881E00E94840889B38F70182B39
:1011800080E00E948408812F99271F91089580E0B4
:101190000E949508982F80915901882331F497FD7A
:1011A00004C0892F8F7780935A01892F992787FD53
:1011B00090958827990F881F992708959B01AC0166
:1011C0008091400390914103A0914203B091430369
:1011D00082179307A407B507A0F080914003909170
:1011E0004103A0914203B0914303821B930BA40BD4
:1011F000B50B80509041A040B040A0F080E090E05E
:1012000008958091400390914103A0914203B091D1
:101210004303281B390B4A0B5B0B2050304F4F4FB9
:101220005F4F18F081E090E0089580E090E008952D
:101230000895EF92FF920F931F93AA27BB27E09088
:101240004003F09041030091420310914303E80EE4
:10125000F91E0A1F1B1F01C0A895C801B7010E94F3
:10126000DE088823C9F31F910F91FF90EF90089536
:101270000F931F93CF93C82F162F042F80916500D3
:101280008D7F8093650080E00E9484088AB38F6020
:101290008ABB8BB3807F9C2F92959F70892B8BBBD1
:1012A000112321F080916500816003C08091650069
:1012B0008E7F8093650081E00E94840880E00E9418
:1012C0008408002329F088E090E00E9419090DC0ED
:1012D0008BB3807FCF708C2B8BBB0E947F0881E00B
:1012E0000E948408802F0E948408CF911F910F9143
:1012F00008950F931F93CF9388E290E00E941909FD
:1013000041E060E080E30E94380941E060E080E372
:101310000E94380941E060E080E30E94380941E022
:1013200060E080E20E94380988E20E94490C80E473
:101330000E94490C8AE00E941A0C89E20E94490C22
:101340008CE10E94490C82E50E94490C89E60E94CA
:10135000490C84E70E94490C80E40E94490C85E115
:101360000E941A0C88E20E94490C80E40E94490CF9
:101370000E94C10E8C0101C0A895909144038091F8
:1013800045039817C9F70E94C708C82F8823A1F7FB
:1013900081E00E9495088A3021F481E0F80184A759
:1013A00002C0F801C4A788E00E94490C81E00E94B5
:1013B000490C86E00E94490C8CE00E94490C60E0D8
:1013C000862F0E94530C67EB71E080E00E94820D33
:1013D0006FE871E081E00E94820D67E971E082E0D0
:1013E0000E94820D6FE771E083E00E94820DCF9131
:1013F0001F910F9108951F920F920FB60F92112413
:101400002F933F934F935F936F937F938F939F930C
:10141000AF93BF93CF93EF93FF93809158018823AD
:1014200009F08FC081E08093580178948091560133
:101430008F5F809356018091560183709927813088
:101440009105F9F0823091051CF4892B21F077C0C9
:10145000039759F174C08091400390914103A0918A
:101460004203B09143030196A11DB11D8093400337
:1014700090934103A0934203B09343030E94E50B72
:101480005EC08091400390914103A0914203B091CE
:10149000430381709070A070B070892B19F00E9486
:1014A000510B4DC00E94120B4AC060915701662338
:1014B00019F00E94C70841C09091440380914503F0
:1014C000981789F0C0914503EC2FFF27EC5BFC4F88
:1014D0002281CF5FC03108F0C62F203829F58091D6
:1014E00044038C1719F480E090E027C0EC2FFF270D
:1014F000EC5BFC4F22812F3F19F420915A012068A8
:1015000027FF02C060935901822F9927807C907039
:101510008034910519F481E080935901CF5FC03187
:1015200008F0C62F462F02C0462F61E0822F0E948E
:101530003809C093450381E090E0809357011092F1
:101540005801FF91EF91CF91BF91AF919F918F91F2
:101550007F916F915F914F913F912F910F900FBEAF
:101560000F901F90189510927D0080B7877F80BFE5
:1015700017BE11BE89E683BF82E085BD87B7806450
:1015800087BF0895EF92FF920F931F93AA27BB275F
:10159000E0904003F0904103009142031091430317
:1015A000E80EF91E0A1F1B1F02C00E94F805C801A1
:1015B000B7010E94DE088823C1F31F910F91FF90AD
:1015C000EF900895282F220F61112160822F8370E0
:1015D0008150823028F424FF02C02E6001C0217F98
:1015E000822F9927089590915D01E92FFF27E35AF3
:1015F000FE4F8283892F8F5F80935D01883010F0CA
:1016000010925D0190915E0180915D01981741F407
:10161000892F8F5F80935E01883010F010925E01F9
:10162000089508950F931F9311B1812F8074682F2F
:1016300080915B010E94E20A082F80935B01107881
:10164000612F80915C010E94E20A80935C01007C22
:10165000807C003829F4882339F0803C61F408C08C
:10166000003449F4803C11F489E103C0882319F463
:101670008AE10E94F30A1F910F910895893118F0B1
:1016800080E090E0089520E030E0E82FFF27E9595E
:10169000FE4F8081882311F021E030E0C9010895D8
:1016A0000895FF920F931F93CF930E94F405182F74
:1016B00080918601181729F01093860182E20E941A
:1016C000F30A80918501E82FFF27E058FE4F008143
:1016D00013B31F7081B1880F880F8071182B10838E
:1016E000FF248091850125E0829FF0011124EF0DF8
:1016F000F11DEA54FF4FC49110FD31C000FF14C02A
:10170000C63129F485E10E943E0B882331F48C2FE9
:101710000E94F30AC93108F043C0EC2FFF27E959B2
:10172000FE4F81E080833CC0C931D0F5EC2FFF270C
:10173000DF01A959BE4F9C919F5F9C93992311F49F
:101740009F5F9C937597329758F580917C018937FC
:1017500038F180917D01893718F1822F1FC0C9317E
:1017600028F4EC2FFF27E959FE4F108200FD18C026
:101770008C2F80680E94F30A0E94F405853081F462
:10178000C53121F486E10E943E0B05C0C63141F40B
:1017900085E10E943E0B882319F486E00E94CC0567
:1017A00016950695F39484E08F1508F09ACF8091F2
:1017B00085018F5F80938501853010F0109285013F
:1017C000CF911F910F91FF900895909185019430D2
:1017D00029F485B3806F85BB97980895979A85B350
:1017E0008F7020E130E002C0220F331F9A95E2F79C
:1017F000922F9095907F892B85BB089508958091B5
:101800005D0120915E01821719F48FEF9FEF08951B
:10181000E22FFF27E35AFE4F8281482F5527822F60
:101820008F5F80935E01883010F010925E01CA01D4
:1018300008950895CF93C82F07C08091450388234A
:1018400091F40E948525A89580914403282F332781
:1018500080914503992701972817390791F38091C3
:1018600044038F3051F3F89480914403E82FFF270D
:10187000EC5BFC4FC283809144038F5F80934403F1
:1018800080914403803110F0109244037894CF91FA
:1018900008951F93182F80E80E941A0C812F0E9430
:1018A0001A0C1F9108958295880F880F807C860FEF
:1018B00080680E94490C08950E94530C8EE00E949B
:1018C000490C08958CE00E94490C0895FF920F93F3
:1018D0001F93CF93F82E60916703809166030E9457
:1018E000530CC0E006E513E080916803C81778F454
:1018F000FF2021F0F80161918F0101C060E282E0D8
:101900000E94AA0DCF5F80916803C81788F3CF911A
:101910001F910F91FF90089590937103809370032E
:10192000892B89F170936F0360936E03CB01AA2713
:10193000BB272091400330914103409142035091D5
:101940004303280F391F4A1F5B1F20936A033093FC
:101950006B0340936C0350936D03809169038E7FFA
:1019600080936903211531054105510561F42F5F0D
:101970003F4F4F4F5F4F20936A0330936B03409369
:101980006C0350936D0308950895AF92BF92CF9268
:10199000DF92EF92FF920F931F93CF93DF93D82E96
:1019A000C62EEA0186E5E82E83E0F82E1092710338
:1019B0001092700381E08D1568F1EFE0E61750F1A9
:1019C0004115510539F1FA0101900020E9F73197ED
:1019D0000E2F041B013108F000E16C2D8D2D0E94AB
:1019E000530C5701002361F0102F8881F50181937A
:1019F0005F018991682F82E00E94AA0D1150A9F71A
:101A0000F701D08AC18A028B64EF71E086E69CE020
:101A10000E948C0CDF91CF911F910F91FF90EF905E
:101A2000DF90CF90BF90AF900895CF93DF93CDB765
:101A3000DEB7A0970FB6F894DEBF0FBECDBF282F3C
:101A4000DE01119690E0FA014F5F5F4F8491882389
:101A500021F08D939F5F9F31B0F31C92AE014F5FD9
:101A60005F4F822F0E94C50CA0960FB6F894DEBF80
:101A70000FBECDBFDF91CF910895809170039091FB
:101A80007103892BA9F160916A0370916B038091B6
:101A90006C0390916D030E94DE08882349F18091C8
:101AA0006903E0917003F091710381700995809151
:101AB000690391E089278093690380916E03909177
:101AC0006F039C0144275527809140039091410367
:101AD000A0914203B0914303820F931FA41FB51F2F
:101AE00080936A0390936B03A0936C03B0936D0390
:101AF00008950895109271031092700381E00E947E
:101B0000490C08950F931F93CF93DF93EB01883017
:101B1000B8F4992723E0880F991F2A95E1F780648C
:101B20000E94490C07E010E0FE01219684910E947A
:101B30001A0C0150104017FFF7CF8FEF0E94490C8D
:101B4000DF91CF911F910F910895813308F080E3C9
:101B500081BF0895CF93C62F9927009709F456C0E7
:101B6000029709F056C067FF4DC00E94C10EFC01EC
:101B700084A58823C1F0C43E11F4C4E843C0C63F25
:101B800011F4C4E93FC0CC3F11F4C1E83BC0C43CF0
:101B900011F4CEE837C0C63D11F4C9E933C0CC3DDD
:101BA00049F5CAE92FC0C43E11F4C1EE2BC0C63FAF
:101BB00011F4CFEE27C0CC3F11F4C5EF23C0C43CD5
:101BC00039F467EE70E084E00E94820DC4E01AC030
:101BD000C63D39F46FED70E085E00E94820DC5E0EE
:101BE00011C0CC3D39F467ED70E086E00E94820DB3
:101BF000C6E008C0CF3D31F46FEC70E087E00E9492
:101C0000820DC7E08C2F0E941A0C03C0862F0E9401
:101C1000672CCF9108951F93CF93DF93182FEB017B
:101C2000FB016491662349F0812F0E94AA0D219641
:101C3000FE018491682F8823B9F7DF91CF911F911E
:101C400008951F93CF93DF93182FEB01888188238A
:101C500041F08991682F812F0E94AA0D88818823E5
:101C6000C1F7DF91CF911F9108951F93CF93DF9319
:101C7000CDB7DEB7C055D0400FB6F894DEBF0FBE6B
:101C8000CDBF67961FAD679769968EAD9FAD69977B
:101C9000AE01475A5F4FBC01CE0101960E946E2FE4
:101CA000BE016F5F7F4F812F0E94210EC05BDF4F0F
:101CB0000FB6F894DEBF0FBECDBFDF91CF911F915D
:101CC00008951F93CF93DF93CDB7DEB7C055D040B3
:101CD0000FB6F894DEBF0FBECDBF67961FAD6797F6
:101CE00069968EAD9FAD6997AE01475A5F4FBC01B3
:101CF000CE0101960E94972FBE016F5F7F4F812F0B
:101D00000E94210EC05BDF4F0FB6F894DEBF0FBEFE
:101D1000CDBFDF91CF911F9108959927009729F0AA
:101D2000029731F40E94FF0B08950E94952C0895AC
:101D30008FEF9FEF08950895E82FFF27EF70F07061
:101D4000E95EFD4F849199270895992783709070DB
:101D50008330910534F48130910534F4892B51F0AE
:101D60000CC0039721F009C084E090E008958EE054
:101D700090E008958FE090E0089584E090E0089569
:101D8000089587E891E0089580919F0182FF05C042
:101D90008091890190918A010895809187019091A5
:101DA00088010895089590919F0192FF05C0809148
:101DB0007203823029F0089580917203873069F4AC
:101DC000109272039260977F90939F011092A201EC
:101DD00060E070E0CB010E948C0C089508950F9391
:101DE0001F93CF93DF93C7E8D1E080919F0199279C
:101DF0008C010170107080FF03C080E090E021C072
:101E000060918F0170919001809191019091920168
:101E1000611571058105910531F00E94DE08882366
:101E200011F4C8010EC01A821B821D8E1E8E1092E4
:101E3000880110928701188E1F8E0E94C80581E0CC
:101E400090E0DF91CF911F910F9108951F93CF9351
:101E5000AC01C62F11E080919F018C7F80939F0180
:101E60001092A5011092A4016623F1F56093A601DA
:101E700020918701309188012115310521F030939F
:101E80008C0120938B0110928A011092890110928B
:101E90008E0110928D011092880110928701C093DB
:101EA000A001C09372034115510559F1BA018FEF9A
:101EB0000E94CA2380919F019927969587959C013E
:101EC0002170307080FD1DC030938A0120938901FC
:101ED00030938E0120938D013093880120938701E8
:101EE000C093A0011C2F0DC0109272036091870156
:101EF000709188018FEF0E94F92380919F0181FFEB
:101F000010E080919F018B7F8260E7E8F1E0808F95
:101F1000812F9927CF911F9108951F93182F6CE05F
:101F200080E00E94530C1123C1F08091A2019927F7
:101F30008F7790709F938F9387E292E09F938F9318
:101F400082E08F930E94610E80E00E941A0C0F9035
:101F50000F900F900F900F9005C06BE272E082E03F
:101F60000E940B0E1F9108959C0180918901909110
:101F70008A01892B11F4C90108952F703F7B77FDE9
:101F80003064CB018F70907044E0880F991F4A95A0
:101F9000E1F7822B932B08950895FC01809187012E
:101FA000909188012091890130918A01E817F90701
:101FB000F9F46093A101232BB1F080918D019091F0
:101FC0008E01F4E096958795FA95E1F7BC016F7064
:101FD0007070892F99278695869580FD7068CA0153
:101FE0000E94B40F11C050938E0140938D0110C018
:101FF000E217F30779F46093A101BA0180918D0192
:1020000090918E010E94B40F90938E0180938D0168
:102010000E94C80508950895FC01CA01309769F42B
:1020200010929F0110928F011092900110929101D5
:10203000109292010E94EF0E089520919F01422F6D
:10204000552741FD2FC06093A10190938E0180938D
:102050008D018091400390914103A0914203B09182
:10206000430388519C4FAF4FBF4F816080938F01D6
:1020700090939001A0939101B093920142FF09C007
:1020800021602B7F20939F01F0938A01E0938901C7
:1020900007C02E7F20939F01F0938801E093870172
:1020A0000E94C8050895089520919F0121FD14C044
:1020B0002B7F216020939F0190938A018093890157
:1020C00080918D0190918E010E94B40F90938E01AA
:1020D00080938D010E94C80508950895CF93DF93E2
:1020E000EB018093A0010E949C0E8093A301209796
:1020F00059F046EA51E060E070E0CE010E94292AE2
:10210000D093A501C093A4010E94C805DF91CF918F
:102110000895CF93C82F882329F06FE471E083E0FE
:102120000E94820DCC2319F067E471E002C06FE6D3
:1021300071E084E00E94820DCC2319F06FE371E01E
:1021400002C067E671E085E00E94820DCC2319F0A1
:1021500067E371E002C06FE571E086E00E94820DE6
:10216000CC2319F06FE271E002C067E571E087E00F
:102170000E94820DCF910895CF93DF93C82FDD2762
:10218000C4FF02C083E001C085EA0E941A0CC0FFB0
:1021900002C084E001C085EA0E941A0CC1FF02C09F
:1021A00085E001C085EA0E941A0CC2FF02C086E0E9
:1021B00001C085EA0E941A0CC3FF02C087E001C07B
:1021C00085EA0E941A0CDF91CF9108958093B201A5
:1021D0000E94C8050895882319F06FE071E002C0DD
:1021E00067E171E082E00E94820D089508958823DE
:1021F00019F06FE171E002C067E271E081E00E94D6
:10220000820D089508950F931F93CF9307E811E06F
:10221000C091B201CC2399F060E081E00E94530CA0
:102220008C2F81500E94AA22BC0182E00E940B0EDA
:102230001092B20188EE93E00E94C20A02C0882385
:1022400019F00E947A0D03C0682F0E94530C8091F0
:10225000870190918801892BF9F00E942823FC01C5
:10226000828193814091870150918801841795075D
:1022700049F4218532858091A4019091A501281708
:10228000390751F0428353838091A4019091A501B5
:10229000818792870E94CD22209187013091880109
:1022A0002115310531F4F80126833783128E138E00
:1022B000118E80919F0182FD0DC080919B019091B4
:1022C0009C01A0919D01B0919E010097A105B105CF
:1022D00019F105C060E372E082E00E940B0E80916C
:1022E0009B0190919C01A0919D01B0919E01BF9393
:1022F000AF939F938F9383E392E09F938F9382E0BA
:102300008F930E94610E8DB79EB707960FB6F89413
:102310009EBF0FBE8DBF4AC02115310531F466E462
:1023200072E082E00E940B0E18C03F932F938DE461
:1023300092E09F938F93C2E0CF930E94610E8091B1
:102340009F010F900F900F900F900F9080FF02C091
:102350008C2F01C080E20E941A0CC091A0010E9443
:10236000F405282F863008F02150233091F4809115
:10237000870190918801892B61F08C2F99278370B8
:10238000907023E0880F991F2A95E1F781549E4FA2
:1023900009C0822F992703E0880F991F0A95E1F75A
:1023A00081529E4FBC0182E00E940B0E6CE080E0E7
:1023B0000E94530C80919F0183FF0AC08091A2016B
:1023C00099278F7790709F938F9382E592E009C051
:1023D0008091A10199278F7790709F938F9386E5C5
:1023E00092E09F938F9382E08F930E94610E0F90F3
:1023F0000F900F900F900F9080918701909188011E
:10240000892B91F08091A00199278370907001979A
:1024100079F487E10E943E0B882331F080E00E942E
:102420001A0C67EF70E010C080E20E941A0C0FC017
:1024300080E00E941A0C8091A10187FF03C067EB26
:1024400071E002C06FEA71E080E00E94820D0E949C
:10245000F405C82F813049F489E00E947522AC014F
:1024600060E08C2F0E94150D11C180919F0199276A
:1024700013E0969587951A95E1F7AC01417050707D
:1024800080FD04C060E0862F0E94C50C10E08091A2
:102490009F0187FF0DC08091890190918A01892B4E
:1024A00031F48091A0010E94A50E853008F011E062
:1024B00060E081E00E94530C80919B0190919C010F
:1024C000A0919D01B0919E010097A105B10509F46D
:1024D00042C08DE00E943E0B882329F48EE00E94CA
:1024E0003E0B882381F18AE592E09F938F93C2E0AF
:1024F000CF930E94610E8DE00E943E0B0F900F90D3
:102500000F90882379F06FE171E081E00E94820DE5
:1025100067E171E08C2F0E94820D6CE271E087EF21
:1025200090E10EC067E271E081E00E94820D6FE0F1
:1025300071E08C2F0E94820D6CE271E08BEE90E1D5
:102540000E948C0CA3C087E00E947522BC0182E02F
:102550000E940B0E44C08091890190918A010097DE
:1025600069F19F938F9386E692E09F938F9382E029
:102570008F930E94610E80918D0190918E01C4E035
:1025800096958795CA95E1F7C82FCF70892F99271F
:10259000869586950F900F900F900F900F9080FD6D
:1025A000C0618C2F0E94BC10112321F08CE30E948B
:1025B0001A0C15C080E20E941A0C13C086EA91E042
:1025C0009F938F938BE692E09F938F9382E08F93FC
:1025D0000E94610E0F900F900F900F900F9011239B
:1025E00061F48091930190919401A0919501B09133
:1025F00096010097A105B105A9F1809189019091FB
:102600008A01892B79F58091A0010E94A50E853061
:1026100048F160E081E00E94530C86E40E941A0CAD
:10262000C0E001E010E080918D0190918E01802347
:102630009123892B41F0C93018F48C2F8F5C04C092
:102640008C2F865001C085EA0E941A0CCF5F000FC4
:10265000111FCE3040F380E20E941A0C81E00E94EC
:10266000891014C0C0918D01CF7080918D0190911F
:102670008E0197FDC0618C2F0E94BC1080E00E94EB
:1026800089106FE771E083E00E94820DCF911F9166
:102690000F910895EF92FF920F931F93CF93DF93C3
:1026A000CDB7DEB726970FB6F894DEBF0FBECDBF0D
:1026B0008C0186E0FE01319611928A95E9F7F801C6
:1026C00024893589468957896281738121153105AD
:1026D0004105510509F45AC06115710569F1E080A1
:1026E000F180C701AA27BB2782179307A407B50764
:1026F00041F0CB01AA27BB2782179307A407B50790
:10270000D9F4F801808D8E7F808F80818F778983C7
:10271000EE0CEF2CEE1CFF08F1948E2D8F778A8340
:10272000AE014F5F5F4F65E080E00E940026F80138
:102730001282138210821182D8018D919C919C018A
:1027400044275527F80184899589A689B7892817D0
:1027500039074A075B0731F4808D91E089278B7F29
:10276000808F1BC060E081E00E94530C80E00E94DB
:102770007522BC0182E00E940B0EF801808D8470EE
:10278000682F848995890E94260F06C0672B21F443
:10279000F801808D8460808FF801148A158A168A6A
:1027A000178A26960FB6F894DEBF0FBECDBFDF9115
:1027B000CF911F910F91FF90EF90089560918F013D
:1027C0007091900180919101909192016115710534
:1027D0008105910561F00E94DE08882341F0109286
:1027E0008F011092900110929101109292016091CC
:1027F00093017091940180919501909196016115DA
:1028000071058105910571F00E94DE08882351F061
:1028100010929301109294011092950110929601DA
:102820000E94C8056091970170919801809199016B
:1028300090919A01611571058105910561F00E94E1
:10284000DE08882341F010929701109298011092AF
:10285000990110929A0108950895AF92BF92CF9274
:10286000DF92EF92FF920F931F93CF93DF93CDB739
:10287000DEB72C970FB6F894DEBF0FBECDBFBC01FC
:1028800047E8A42E41E0B42E86E0FE013196119275
:102890008A95E9F765317105DCF46F3071050CF04C
:1028A00019C26A30710509F432C36B3071053CF40A
:1028B0006115710509F49BC277FD39C3E3C26C3021
:1028C000710509F443C16D3071050CF097C116C351
:1028D0006B31710584F46931710514F56631710548
:1028E00009F437C2663171050CF473C267317105A2
:1028F00009F4ECC01CC36F3871056CF46D387105B8
:102900000CF07CC16A38710509F4FDC26C387105A0
:1029100009F4F9C20CC36739710509F406C307C38A
:1029200080919F0183FF03C01091A20102C010910A
:10293000A101EE246931710511F431E0E32EF0902C
:10294000A3010E942823FC0107810E942823FC0187
:10295000808184FF33C017FD05C080E0EE2009F4BC
:1029600081E0E82EEE2051F5812F99278F77907026
:10297000892B79F48091970190919801A091990108
:10298000B0919A010097A105B10519F480E81827C4
:1029900062C08091400390914103A0914203B091A5
:1029A0004303845D9E4FAF4FBF4F80939701909339
:1029B0009801A0939901B0939A0118C0EE20B1F04C
:1029C0000E94F405412F5527833041F49A012F7757
:1029D00030708F2D99272817390714F09A0169C094
:1029E000FEE7FF1651F5002371F427C0212F33278E
:1029F000C9018F779070892B09F45BC08EE7F816B8
:102A000049F5002339F160E8462F013011F440E028
:102A100009C0023019F444E16EE304C0033011F43C
:102A20004AE066E1EE2059F0812F99278F77907068
:102A3000242F33278217930714F41F5F0CC0EE2056
:102A400069F4812F99278F779070242F33272817C7
:102A5000390724F01150212F33272BC0812F9927BC
:102A60008F779070462F5527481759071CF0212F54
:102A70002E7F04C0212F261B2C7F260F211711F03B
:102A8000EE20B1F03327EE2051F0C9018F7790701E
:102A90008417950714F02C5F0BC02E5F09C0C90185
:102AA0008F7790704817590714F4245001C02250B2
:102AB0003327122F80919F0183FF05C0F501238FDB
:102AC0001078128F32C2F501228F2FC290919F0190
:102AD00097FF26C088E0892780939F01992723E0EC
:102AE000969587952A95E1F79C012170307080FFBB
:102AF0000CC08091A1018093A20180788093A101F4
:102B000060E971E08DE89FE008C08091A2018093A8
:102B1000A1011092A201B901C9010E948C0C05C249
:102B20008091A001992783709070019729F467EF35
:102B300070E080E00E94820D8091A10180958078F4
:102B40008093A10180919F01877FEDC1C090890191
:102B5000D0908A01C114D104E9F5E0909B01F09076
:102B60009C0100919D0110919E011E141F041006EE
:102B7000110684F58091A0010E94A50E9927AA272D
:102B8000BB278E159F05A007B10724F180919B01FB
:102B900090919C01019721E030E002C0220F331F89
:102BA0008A95E2F780918D0190918E01822793277B
:102BB00090938E0180938D0180919F018068809316
:102BC0009F0110929B0110929C0110929D01109206
:102BD0009E01ABC180919F0187FF09C0CD2839F0CC
:102BE00080918D0190918E0120E030E4ACC0809105
:102BF0008D0190918E0120E030E8A5C086E097E03D
:102C0000E92EF12CEC0EFD1EF70111928A95E9F7E1
:102C100080919B0190919C01A0919D01B0919E019A
:102C20000097A105B10509F453C000919B011091D3
:102C30009C0101501040000F111FCB018F77907045
:102C40000E9709F4016067FF28C01A8680919F01E2
:102C50009927B3E096958795BA95E1F79C01217085
:102C6000307080FD03C0B901C90104C060E971E0A2
:102C70008DE89FE00E948C0C6FE871E081E00E947B
:102C8000820D67E971E082E00E94820DE7E8F1E0E1
:102C9000148A158A168A178A02C081E08A87802FD3
:102CA0008F778F83000F012F001F110B1195802F3D
:102CB0008F778887000F012F001F110B1195802F30
:102CC00083708987A70166E080E00E9400262DC1FD
:102CD00067FD2BC1613171050CF1809189019091E3
:102CE0008A01892B09F021C18091A0019927837065
:102CF00090700197029708F418C180914003909159
:102D00004103A0914203B09143038C509E4FAF4FBB
:102D1000BF4FF50184879587A687B787962F9D506B
:102D200080919F0187FF04C0613171050CF49C5FA5
:102D300021E030E002C0220F331F9A95E2F7809124
:102D40008D0190918E0182279327F50186839783C9
:102D5000ECC0850180919B0190919C01A0919D0107
:102D6000B0919E010097A105B10589F180919F0165
:102D700082FD2DC00E94F405833019F58091A301D6
:102D8000282F33274427552780919B0190919C0140
:102D9000A0919D01B0919E01281739074A075B0752
:102DA00044F420939B0130939C0140939D015093E8
:102DB0009E018091A101807890919B01892B809345
:102DC000A101F801148A158A168A178AAEC043E059
:102DD00005C080919F0187FF04C042E060E280E06F
:102DE00003C040E060E2842F0E9423299EC08091AE
:102DF0009F0187FF12C080918B0190918C010097F9
:102E000009F495C0AA27BB2780939B0190939C014E
:102E1000A0939D01B0939E011EC082FF20C08091AF
:102E20009B0190919C01A0919D01B0919E01009702
:102E3000A105B105A1F486E00E943F2280919B018B
:102E400090919C01A0919D01B0919E010097A105D8
:102E5000B10509F46CC0C5010E944A1368C0809195
:102E60009B0190919C01A0919D01B0919E010097C2
:102E7000A105B10539F48FEF0E943F2281E00E9445
:102E8000031155C080919B0190919C01A0919D01DF
:102E9000B0919E019C01AD01E3E0220F331F441F5E
:102EA000551FEA95D1F7280F391F4A1F5B1F280FBE
:102EB000391F4A1F5B1FCB01AA2797FDA095BA2F88
:102EC000280F391F4A1F5B1F2030F8E23F07F0E050
:102ED0004F07F0E05F0724F080919F0186FF27C035
:102EE000203080E4380780E0480780E05807FCF491
:102EF000F501248B358B468B578B17C087E891E003
:102F00000E944A1312C080919F018F770CC01092CB
:102F10009B0110929C0110929D0110929E01809144
:102F20009F018B7F806880939F010E94C8052C962B
:102F30000FB6F894DEBF0FBECDBFDF91CF911F91CA
:102F40000F91FF90EF90DF90CF90BF90AF900895DA
:102F5000FB0121E057FF04C020E0509541955F4FF1
:102F60008330910549F18430910534F48130910525
:102F700091F0029729F12AC08430910519F0059744
:102F800061F024C081818F5F818399278417950721
:102F9000ECF0222359F0118219C081818150818384
:102FA00099278417950794F0222321F0842F8150CC
:102FB00081830CC021830AC012821382168A06C044
:102FC00090E08281882309F491E0928380E090E090
:102FD00008950F931F93CF93DF938C010E94C40E2B
:102FE000EC01009731F469E476E082E00E940B0E78
:102FF0000FC09F938F938FE496E09F938F9382E00F
:103000008F930E94610E0F900F900F900F900F9072
:103010000115110521F0B80182E00E940B0ECE01CE
:10302000DF91CF911F910F9108950F931F93CF932D
:10303000DF93FC018B01EA0180819181892B31F0C2
:10304000818D992783709070039779F060E081E01B
:103050000E94530C85E00E947522BC0182E00E9410
:103060000B0E0330110519F11FC00E94F4058330C7
:10307000F1F00E94F4058230D1F00630110531F4F0
:1030800043E060E280E00E9423290EC060E081E01E
:103090000E94530C86E00E947522BC0182E00E94CF
:1030A0000B0E1A821B821E8A80E090E002C081E033
:1030B00090E0DF91CF911F910F9108951F93182FEA
:1030C0000E94C10EFC01808D112311F0806401C0AB
:1030D0008F7B808F1F9108950F931F93CF93DF9362
:1030E000EC018B01009731F097FD35C002970297F4
:1030F00090F52BC060E081E00E94530CF8018281C2
:10310000882359F463E576E082E00E940B0E6CE5BB
:1031100076E082E00E940B0E18C00E944C23DC0176
:10312000CB01BF93AF939F938F9382E696E09F93DB
:103130008F9382E08F930E94610E8DB79EB70796A2
:103140000FB6F8949EBF0FBE8DBF40E050E0B801AF
:10315000CE010E94A81780E090E0DF91CF911F91EF
:103160000F9108958230910541F08330910541F42B
:1031700040E050E00E94A81703C08FEF9FEF089532
:1031800080E090E0089508952F923F924F925F92D1
:103190006F927F928F929F92AF92BF92CF92DF9267
:1031A000EF92FF920F931F93CF93DF93CDB7DEB7CC
:1031B00026970FB6F894DEBF0FBECDBF8C016B0112
:1031C0000E94C10E7C010230110509F480C0033059
:1031D00011053CF40115110519F10130110531F00B
:1031E00012C1063011050CF00EC132C0FC01118D68
:1031F000212F2695269523701370808D86FF04C09D
:10320000112311F414E003C0112309F411E083E049
:10321000189FC0011124280F2350F6012183F3C009
:1032200060E081E00E94530C8EE696E00E94E91770
:10323000892B09F4E8C0F60191818AE0989FC001CA
:1032400011248B559D4FBC0182E00E940B0EDBC008
:10325000FC01808D86FF03C04AE050E002C049E0D7
:1032600050E0B601C8010E94A817F7018081918142
:103270008F3F9105B9F0B0F0F6018181882311F4F8
:1032800086E08183F701808D86FD06C0F60181818D
:10329000863010F488E08183F6018181863010F455
:1032A00089E08183F701808191818050984208F400
:1032B000AAC0F6018181882311F489E08183F60197
:1032C0008181893008F09FC089E081839CC0FC0126
:1032D000628073806114710409F095C0F6018281E7
:1032E000882309F488C0F7018080918081149104BB
:1032F00009F489C0818D0E949C0E5C01F601218138
:10330000822F63E00E94B332182F1F5F822F0E942A
:10331000B332892F9927880F991F880F991F182B6F
:10332000143009F410E0F701258C368C812F0E94AF
:103330009C0EF701428D242F33272F773070289F62
:10334000B001299F700D389F700D1124CB01B5017C
:103350000E94BF324078462B428F4FE1442E512CC1
:103360004E0C5F1C3AE0A32EB12CAC0CBD1CB2017C
:10337000C5010E94672F86E0FE01319611928A9561
:10338000E9F7882D8F778983C401880F892F881FDB
:10339000990B91958F778A831F771B83AE014F5FBF
:1033A0005F4F64E08FEF0E94002660E081E00E94A2
:1033B000530C80E00E947522BC0182E00E940B0E3B
:1033C000A30160E0C3010E940C10B4018FEF0E94C2
:1033D000CA232114310459F09501F701418D608110
:1033E0007181C1010E946C29F701858F968FB5010B
:1033F000C2010E94672F90E0F6018281882309F4C0
:1034000091E0F601928380E090E026960FB6F89462
:10341000DEBF0FBECDBFDF91CF911F910F91FF9007
:10342000EF90DF90CF90BF90AF909F908F907F9064
:103430006F905F904F903F902F900895482F30E00D
:10344000832F992787FD9095FC01EC58FD4F24911F
:10345000241729F03F5F222399F78FEF9FEF0895FC
:103460000895EF92FF920F931F93CF93DF93EB0199
:103470008230910509F486C08330910534F40097B9
:1034800009F43EC0019769F0BAC08430910509F48F
:1034900043C0843091050CF470C0059709F456C000
:1034A000AEC00E94C10E8C01FC0180819181892BEC
:1034B00009F4A5C06FE1E62EF12CE00EF11E8E019D
:1034C000065F1F4F65960C171D07B8F4F701808142
:1034D000882339F00E941E1A87FD03C0F7018081FE
:1034E00001C080E2F80181938F01F7018081882378
:1034F00051F30894E11CF11CE6CFF80110827FC063
:103500000E94E91760E081E00E94530C2A96BE01F8
:1035100082E00E94210E73C08981FB01E80FF11D3A
:10352000EF012A9682850E941E1A8F5FE82FFF27DF
:10353000E7FDF095EC58FD4F8491882319F4E4E7FA
:10354000F2E08491992787FD909515C08981FB0150
:10355000E80FF11DEF012A9682850E941E1A1816A7
:1035600014F08FE201C08150E82FFF27E7FDF095AE
:10357000EC58FD4F8491888342C04AE050E00E949D
:10358000A8173DC00E94C10E8C01FC01828193816D
:10359000892BA9F59A81992349F489E08B8381E0ED
:1035A000888F99839F8B8A838E8B29C089818F5FB7
:1035B00089838F8B8B3018F11B821A821E8A8CE0D4
:1035C0009801215E3F4FD901FE013A9601900D927C
:1035D0008A95E1F7F801858D968D009731F0418D40
:1035E000608171810E946C2907C0A901F801618D79
:1035F000808191810E94212AF801858F968F80E039
:1036000090E0DF91CF911F910F91FF90EF9008957F
:103610006F927F929F92AF92BF92CF92DF92EF9282
:10362000FF920F931F93CF93DF93CDB7DEB727970A
:103630000FB6F894DEBF0FBECDBF9C018B01823068
:10364000910509F455C0833091052CF40097C1F021
:10365000019759F0E9C084309105D9F18430910582
:103660000CF441C00597C9F1DFC04BE050E060E2C7
:1036700070E0C8010A960E94602FF801158AD4C034
:10368000FB018281882309F4CFC08181882309F45A
:10369000CBC0065F1F4FA801B90199270E94292AB4
:1036A0009F938F9381E796E09F938F9392E0F92EFB
:1036B000FF920E94610E60E081E00E94530CB8010D
:1036C0008F2D0E94210E0F900F900F900F900F9052
:1036D000ABC0FB018181992721C0FB018181992722
:1036E0000E94172B1DC040E050E00E94A8179CC00C
:1036F00090E0FB018281882309F491E0F801928334
:103700000E94C10E7C01F8019280992061F0FC01B9
:10371000858D968D009711F0858D02C00E94132B28
:10372000F801818381C08AE0682E712C600E711EC1
:10373000F8018181A301BE01695F7F4F99270E9433
:10374000292A5C01F701208D822F9927969587956C
:1037500096958795A1E0CA2ED12CC822D92280FF48
:1037600008C0C501AA27BB27848B958BA68BB78B76
:1037700058C0F70180819181009711F0848395836F
:10378000F701C282D382C682D782C082D1822C7FC7
:10379000208FB5018FEF0E94CA23F70180819181AC
:1037A000892B79F186E0FE01319611928A95E9F72D
:1037B0008A2D8F778983C501880F892F881F990BE0
:1037C00091958F778A838F818F778B83AE014F5F3F
:1037D0005F4F64E08FEF0E940026692D81E00E9418
:1037E000530C892D0E947522BC0182E00E940B0EB1
:1037F000A601692DC6010E940C10B5018FEF0E9431
:10380000CA23F70180819181892B59F0B301C70147
:103810004F960E94672FF80181819927F701858FC4
:10382000968F8FEF9FEF02C080E090E027960FB653
:10383000F894DEBF0FBECDBFDF91CF911F910F91E6
:10384000FF90EF90DF90CF90BF90AF909F907F90D0
:103850006F9008950F931F93CF93DF93EC010E9415
:10386000C10E8C01209719F02297C9F03DC0CE01FE
:103870000E94E917892BC1F160E081E00E94530C9E
:10388000F801858D968D892B11F081E001C082E0D1
:103890000E947522BC0182E00E940B0E25C0FC0133
:1038A000C281D381209701F580819181892BE1F03C
:1038B000858D968D892BC1F060E081E00E94530CCC
:1038C00083E00E947522BC0182E00E940B0E84EF0F
:1038D00091E00E94C20AF801858D968D0E944229CE
:1038E000F801C58FD68F178E80E090E0DF91CF91E1
:1038F0001F910F910895CF93DF93EB0182309105D3
:1039000061F1833091052CF4009781F0019729F043
:1039100034C0863091058CF51BC00E942823FC0121
:1039200087818983843048F1198227C060E081E073
:103930000E94530C8981865F0E9475229F938F930A
:1039400082E08F930E94610E0F900F900F9015C030
:1039500044E050E00E94A81710C08A81882339F003
:103960000E9428232981FC0127830E94CD2290E018
:103970008A81882309F491E09A8380E090E0DF91C6
:10398000CF910895CF93DF93EB018230910589F1B8
:10399000833091052CF40097A9F0019731F043C0D2
:1039A000863091050CF03FC01FC00E942823FC0107
:1039B0008081992724E0969587952A95E1F7817073
:1039C000898331C060E081E00E94530C8981825F6D
:1039D0000E9475229F938F9382E08F930E94610EC5
:1039E0000F900F900F901FC042E050E00E94A81768
:1039F0001AC08A81882389F08981882331F00E9446
:103A00002823FC018081806105C00E942823FC01DD
:103A100080818F7E80830E94CD2290E08A818823DE
:103A200009F491E09A8380E090E0DF91CF910895CE
:103A30001F93CF93DF93EB018230910509F440C0CF
:103A4000833091052CF4009789F0019731F04CC038
:103A5000863091050CF048C02EC00E942823FC013E
:103A6000848163E00E94B33289833EC060E081E0DC
:103A70000E94530C898113E0819F802D11240E94A4
:103A8000A50D82E090E00E94C20A81B7612F0E94DA
:103A9000B332898399279F938F9385E796E09F930D
:103AA0008F9382E08F930E94610E0F900F900F9082
:103AB0000F900F9019C04FEE5FEF0E94A81714C02F
:103AC0008A81882359F00E942823398123E0329F7C
:103AD00090011124FC0124830E94CD2290E08A8170
:103AE000882309F491E09A8380E090E0DF91CF9100
:103AF0001F910895CF92DF92EF92FF920F931F9341
:103B0000CF93DF93CDB7DEB726970FB6F894DEBF1D
:103B10000FBECDBF8C017B010E94C10E6C01A701BD
:103B2000B8010E941518882309F406C10230110556
:103B300009F4A1C0033011053CF40115110539F158
:103B40000130110571F0F8C00430110509F491C07D
:103B5000043011050CF4EAC00530110509F4E2C087
:103B6000EBC08EEF9FEFF701818F928F2091BC0108
:103B70003091BD01C90101978050944020F4F701B4
:103B800024833583D9C0F70104831583D5C0F70199
:103B90008281882309F4D0C060E081E00E94530C48
:103BA000F7018281882309F4C7C060E081E00E94A8
:103BB000530CF701848195819F938F9389E796E059
:103BC0009F938F9312E01F930E94610E0F900F90AE
:103BD0000F900F900F90F7018381843059F48FE795
:103BE00096E09F938F931F930E94610E0F900F900A
:103BF0000F9011C0F701808599279F938F9383E8D9
:103C000096E09F938F931F930E94610E0F900F90E9
:103C10000F900F900F90F701818D928D97FD03C04B
:103C200067E876E00AC08E5F9F4F19F46FE876E090
:103C300004C084E00E947522BC0182E00E940B0E49
:103C400081E0F701808F868B8381992781309105F0
:103C50006CF08330910524F00497029738F402C089
:103C600083E001C088E0F701878B66C0F701168A00
:103C700063C084E058C0F7018281248135818823A4
:103C800089F441E0438380E094E086839783821740
:103C900093072CF481E090E0F70184839583F7018A
:103CA00042834AC03093BD012093BC0121153105E8
:103CB000C9F1F701838181508230A0F1F601808142
:103CC0008F77898380819181880F892F881F990B35
:103CD00091958F778A83F701848181508F778B83C9
:103CE00021503040220F232F221F330B322F3770E9
:103CF0002085822F99278078907095958795382B0D
:103D00003C832F772D831E82AE014F5F5F4F67E0AC
:103D10008FEF0E940026F70113820E94620C8FEF42
:103D20009FEF0CC081E0F701838306C040E050E0C4
:103D3000B701C8010E94A81780E090E026960FB650
:103D4000F894DEBF0FBECDBFDF91CF911F910F91D1
:103D5000FF90EF90DF90CF900895CF92DF92EF9297
:103D6000FF920F931F93CF93DF93CDB7DEB72697C4
:103D70000FB6F894DEBF0FBECDBF7C018B010E9451
:103D8000C10E6C01A801B7010E941518882309F41F
:103D9000C8C042E0E416F10409F48DC083E0E816DF
:103DA000F10444F4E114F10481F1E1E0EE16F104D0
:103DB00089F0B7C0F4E0EF16F10409F456C044E00E
:103DC000E416F1040CF470C085E0E816F10409F47F
:103DD0005AC0A7C08EEF9FEFF801818F928F20917C
:103DE000BC013091BD01C90101978050944020F47D
:103DF000F8012483358303C0F801E482F58280E072
:103E000094E0F801868397838CC0F801828188232F
:103E100009F487C060E081E00E94530CF8018481BE
:103E2000958197FF0CC087E996E09F938F9382E07E
:103E30008F930E94610E0F900F900F900FC09F9371
:103E40008F938CE996E09F938F9382E08F930E94EB
:103E5000610E0F900F900F900F900F9083E0F8017C
:103E6000878B81E0808F868B5CC0F801848195818F
:103E7000019684839583268137818217930784F086
:103E8000248335830DC0F801848195810197848353
:103E900095831816190624F081E090E084839583B9
:103EA00081E0F80183833DC040E050E0B801C701E4
:103EB0000E94A81736C091E0F8019383828188237D
:103EC00071F124813581121613065CF53093BD0122
:103ED0002093BC01F60180818F7789838081918155
:103EE000880F892F881F990B91958F778A83F80106
:103EF000848181508F778B8321503040220F232F74
:103F0000221F330B822F87708C831E821D82AE018D
:103F10004F5F5F4F68E08FEF0E94002602C0F801FC
:103F2000928380E090E026960FB6F894DEBF0FBE35
:103F3000CDBFDF91CF911F910F91FF90EF90DF9058
:103F4000CF900895CF92DF92EF92FF920F931F933D
:103F5000CF93DF937C01C62F0E947A0D0E94282305
:103F60006C01CE3008F070C085E0C89F800111243C
:103F70000E5F1E4FF7018281882311F080E001C09F
:103F800082E00E941A0CF601858199278230910502
:103F900099F0833091051CF4019721F021C003971B
:103FA000A9F01EC08C2F9927C4E0880F991FCA95CD
:103FB000E1F787589A4F1DC08C2F9927B4E0880FDE
:103FC000991FBA95E1F787559B4F13C08C2F9927FE
:103FD000A4E0880F991FAA95E1F787529C4F09C06A
:103FE0008C2F9927F4E0880F991FFA95E1F7875FE6
:103FF0009C4FBC0182E00E940B0EE7016A816623A0
:1040000079F4F801848187FD0BC081E00E94530C94
:10401000E8018C810E947522BC0182E00E940B0E97
:10402000E801EA81FB81309721F0B70180E090E060
:104030000995F7018689882329F06789808D0E9478
:104040005C0C02C00E94620CDF91CF911F910F9116
:10405000FF90EF90DF90CF90089560E0E2E0F1E014
:10406000482F552747FD509520E030E08081992763
:104070008417950711F4C90108956F5F2F5F3F4FB3
:1040800035966D3098F38FEF9FEF08950895BF92A6
:10409000CF92DF92EF92FF920F931F93CF93DF9314
:1040A000CDB7DEB76B970FB6F894DEBF0FBECDBFAE
:1040B000B82E8CE08B1518F480E090E0D0C16E0132
:1040C0000894C11CD11C8BE1F60111928A95E9F785
:1040D000A89585E0B89EF0011124EE5FFE4F0280A6
:1040E000F381E02D309721F0B60181E090E0099551
:1040F0006B2DC6010E94A21F0E94C10E0E94F805EE
:1041000085E0B89E70011124E2E0F1E0EE0EFF1EA2
:104110000E94FF0BAC018531910509F484C1863101
:10412000910574F48A30910509F4DEC08B30910555
:104130001CF497FDE3CFFFC00B9709F48DC0DECFD1
:104140008931910591F08A31910544F486319105C8
:1041500009F472C1479709F47FC0D0CF8A31910525
:1041600039F1829709F475C1C9CFF601828188239C
:1041700081F0F701228133812115310531F0BE0133
:104180006F5F7F4F84E090E062C1F60181818F5FB5
:1041900022C0F601868BF70190816B2D6F5F6D3029
:1041A0001CF48581891729F1892F0E942D203CC09C
:1041B000F6018281882389F0F7012281338121155C
:1041C000310531F0BE016F5F7F4F85E090E03FC168
:1041D000F6018181815081833CC1F601868BF70114
:1041E000908135976B2D615067FD0CC080818917D8
:1041F00049F4772767FD70951BC0842F992787FDA9
:10420000909512C04CE0EEE3F1E0292F332727FD13
:104210003095808199278217930779F3415035971C
:1042200047FFF7CF8FEF9FEF682F772767FD7095D8
:10423000B62E85E0689FF0011124EE5FFE4F0280EC
:10424000F381E02D309709F404C1BE016F5F7F4F09
:1042500081E090E00995FDC0F7019181992361F11A
:10426000092F11270C541E4FF801808118162CF0CD
:10427000892F0E942D20F8018083F7018181E82F8A
:10428000FF27EC54FE4F80810E944720282F3327C0
:1042900027FD3095F7018181E82FFF27EC54FE4F71
:1042A000C90137FF04C088279927821B930B80839D
:1042B00037FFCFC0B1943AC0F70122813381211575
:1042C000310551F0BE016F5F7F4F82E090E0F90150
:1042D000099599237CF319C0F6018281882309F49A
:1042E00091E0F6019283B5C0F60182818823F1F056
:1042F000F7012281338121153105A9F0BE016F5FDD
:104300007F4F83E090E0F9010995F60182818823CF
:1043100009F09FC0F70122813381BE016F5F7F4F9B
:1043200081E090E094C0F601128293C08B2D992712
:1043300087FD909594C0F60183819927843091057B
:1043400009F447C0853091054CF48230910539F16C
:104350008330910584F4019771F07BC0883091051A
:1043600051F0893091051CF40597B9F172C0099795
:1043700009F446C06EC0F60186819781892B21F42D
:104380008FEF9FE786839783F60186819781841755
:1043900095070CF45EC01482158282E08383F601D7
:1043A000848195819C0113E0220F331F1A95E1F758
:1043B000280F391F280F391F240F351F37FD49C01B
:1043C00086819781821793070CF443C02483358339
:1043D00040C0F601108685E08383F60190858AE06F
:1043E000989F90011124240F351F2F3F310509F0AC
:1043F00008F420878EEF9FEFF601818F928F29C0FE
:10440000F6018181E80FF11D842F805D8287F7011D
:104410002281338121153105E1F0BE016F5F7F4FAD
:1044200082E090E014C080E00E94CC0540E060E2B1
:10443000842F0E9423290DC0F70122813381211589
:10444000310539F0BE016F5F7F4F86E090E0F901E2
:1044500009956B2DCE0101960E94A21F4FCE6B963F
:104460000FB6F894DEBF0FBECDBFDF91CF911F9185
:104470000F91FF90EF90DF90CF90BF900895CF9372
:10448000C82F0E945A23803871F16FEE70E080E0EF
:104490000E94820D67EF70E082E00E94820D8091A1
:1044A000B4018D3010F01092B401C7FD04C08C2F00
:1044B0000E9447200EC08091B4010E944720992796
:1044C00087FD909597FF03C0909581959F4F8093AE
:1044D000B40167EB71E080E00E94820D67E971E052
:1044E00082E00E94820DCF910895CF93C82F803132
:1044F00018F084E29BE02CC00E942823FC018581F7
:1045000099278230910581F0833091051CF4019741
:1045100021F018C0039779F015C081E1C89FC00150
:1045200011248C5E954F14C081E1C89FC0011124F5
:104530008C5F964F0DC081E1C89FC00111248C5043
:10454000984F06C081E1C89FC00111248C51994F3A
:10455000CF910895882319F081E39BE008950E948C
:104560002823FC01858199278230910561F08330F1
:1045700091051CF4019721F00CC0039739F009C094
:1045800083ED96E0089582EC96E0089581EB96E045
:10459000089580EA96E008950895EF92FF921F93A0
:1045A000CF93DF938EEBE82E81E0F82EC0E0D0E0D1
:1045B0001FE1CE010E943C2FF70161917F01861718
:1045C00019F0CE010E94552FA8951150219617FF82
:1045D000F0CFDF91CF911F91FF90EF9008959091D0
:1045E000C301973008F091E080E1EEEBF1E0119229
:1045F0008A95E9F788E18093C2019093C3010E94F4
:10460000CD22089540E250E060E070E08EEB91E052
:104610000E94442F8091C0019091C1018F5F9F4FF4
:1046200011F40E94EF228091C301873010F01092A4
:10463000C3018AEF9FEFA1E0B0E0ABBFFC0187911F
:104640008F3F21F0882311F080936F000895089523
:104650008EEB91E008958093C3010E94CD220895CE
:1046600020E030E09091BE01982311F021E030E08D
:10467000C90108959091BE01982B9093BE010E94AC
:10468000CD220895982F90958091BE018923809323
:10469000BE010E94CD2208958CEF9FEFA1E0B0E013
:1046A000ABBFFC0187919791A791B691B070BC0107
:1046B000CD0108958FEF9FEFA1E0B0E0ABBFFC010B
:1046C0008791823011F4079B80E899270895FC01B7
:1046D000808D9927969587959C012170307080FD7B
:1046E00002C0C901089580819181009711F081E095
:1046F00090E008950895FC01808D992796958795FF
:104700009C012170307080FD02C0C9010895828132
:104710009381009711F081E090E008950895CF9281
:10472000DF92EF92FF920F931F93CF93DF93C82EE8
:104730007B01EA01452B29F10E94C10E8C01DD2489
:10474000A7016C2D80E00E94002686E08093730311
:1047500002C00E94F805C801FE010995882321F4D2
:10476000809173038823A9F70E94D1248111DD244D
:10477000C801FE010995882321F4D39489E08D15A1
:10478000F8F6DF91CF911F910F91FF90EF90DF909E
:10479000CF900895CF93DF93CDB7DEB726970FB6AE
:1047A000F894DEBF0FBECDBF61157105C9F086E07C
:1047B000FE01319611928A95E9F7862F8F778983CA
:1047C000660F672F661F770B7195862F8F778A8309
:1047D00047E653E2BE016F5F7F4F81E00E948F2367
:1047E00026960FB6F894DEBF0FBECDBFDF91CF91F6
:1047F0000895CF93DF93CDB7DEB726970FB6F89421
:10480000DEBF0FBECDBF6115710539F141155105F0
:1048100021F186E0FE01319611928A95E9F7862F03
:104820008F778983660F672F661F770B7195862FA9
:104830008F778A83842F8F778B83440F452F441F74
:10484000550B5195842F8F778C834BE753E2BE0134
:104850006F5F7F4F82E00E948F2326960FB6F894F9
:10486000DEBF0FBECDBFDF91CF910895F894FFCF8B
:10487000FC0180E0482F57E02191282780E0922F0B
:1048800096958F5F20FF03C0292F252701C0292F70
:104890008830A8F33327822F4F5F483068F327FD15
:1048A0008095992708950F931F938C010E943824B7
:1048B000F8019085891719F080E090E002C081E04E
:1048C00090E01F910F910895FC01CB01262F2F77C7
:1048D0002083880F892F881F990B91958F7781836B
:1048E0000895EF92FF920F931F93CF93DF93CDB76D
:1048F000DEB729970FB6F894DEBF0FBECDBF9C017F
:104900008091430180687E010894E11CF11C898339
:1049100083E0F701818387010E5F1F4F822F8F771E
:10492000F80181938F01220F232F221F330B319522
:10493000822F8F77F8018193862F8F7781938F0154
:10494000CA01892F9927869586958F73808367FF83
:1049500002C0806480830F5F1F4FCA0133E09695C9
:1049600087953A95E1F78F77F8018193842F8295A7
:10497000807F8F7781938F01C7010E943824F801CF
:104980008083C7010E94470829960FB6F894DEBFBE
:104990000FBECDBFDF91CF911F910F91FF90EF9090
:1049A00008958091E301882319F480E090E0089550
:1049B0001092E30181E090E008950895EF92FF9254
:1049C0000F931F93CF93DF93CDB7DEB729970FB621
:1049D000F894DEBF0FBECDBF0E944C237B018C013B
:1049E00065C0A8958A81843009F060C0CE01019627
:1049F0000E945324882309F459C0D801C7018F7736
:104A00009070A070B0702E813327442755278217ED
:104A10009307A407B50709F049C0D801C7018078FA
:104A20009F73A070B07037E0B595A795979587955F
:104A30003A95D1F72D8133274427552782179307BD
:104A4000A407B50799F5D801C7018070907CAF71B4
:104A5000B0702EE0B595A795979587952A95D1F7D3
:104A60002C8133274427552782179307A407B507BE
:104A7000E9F4D801C70180709070A07EB070F5E1B4
:104A8000B595A79597958795FA95D1F72B813327FB
:104A90004427552782179307A407B50739F489815E
:104AA0008F778093430181E090E007C0CE010196AB
:104AB0000E945108009709F094CF29960FB6F894F8
:104AC000DEBF0FBECDBFDF91CF911F910F91FF9041
:104AD000EF90089520914401309145019093450154
:104AE00080934401C90108959093E1018093E0010E
:104AF00081E08093E2010895E091DE01F091DF0111
:104B0000309709F0099508950895CF93DF93CDB7B5
:104B1000DEB729970FB6F894DEBF0FBECDBF22C017
:104B2000CE0101960E9453248823E1F08A818630C9
:104B300021F481E08093E30115C0809144019091BC
:104B40004501892B31F486E196E2909345018093EB
:104B50004401E0914401F0914501309719F0CE01F4
:104B600001960995CE0101960E945108892BC1F644
:104B700029960FB6F894DEBF0FBECDBFDF91CF915F
:104B8000089580914301992708950F931F93CF9320
:104B9000DF93CDB7DEB729970FB6F894DEBF0FBE0F
:104BA000CDBFFA01A89580914301806889836A830B
:104BB0008E010D5F1F4F95E0309729F081918F771F
:104BC000D8018C9302C0D8011C9291500F5F1F4FE7
:104BD00097FFF2CFCE0101960E943824F80180831E
:104BE000CE0101960E941308992729960FB6F894D2
:104BF000DEBF0FBECDBFDF91CF911F910F91089502
:104C00000F931F93CF93DF93082F162FEA0102C053
:104C10000E94F805AE01612F802F0E94C5258823D0
:104C2000B9F3DF91CF911F910F9108959F92AF92A9
:104C3000BF92CF92DF92EF92FF920F931F93CF9389
:104C4000DF93CDB7DEB726970FB6F894DEBF0FBE61
:104C5000CDBF6C010E94C10E5C01F6012181822F43
:104C600099278C30910509F447C18D309105ACF43A
:104C70008930910554F4873091050CF058C0833089
:104C8000910589F10597C9F152C28A30910509F45D
:104C9000B2C00B970CF0E1C095C08331910509F4C7
:104CA00000C28431910564F48131910509F4CDC1CC
:104CB000823191050CF0E7C1409709F4B4C137C2C5
:104CC0008132910509F424C28232910524F480973F
:104CD00009F41CC22CC28232910509F41EC28397CA
:104CE00009F4F0C124C2F60182810E94CC05F601CC
:104CF000878184700E945E181AC2F6018281082F93
:104D00001127838199279695982F882797958795BE
:104D1000082B192BD5018D919C918017910709F0D3
:104D200006C20E94EF0EC8010E94452D00C2F60186
:104D30008281082F1127838199279695982F88279C
:104D400097958795082B192B8581482F5527542F28
:104D50004427550F550F868199278F77907033E040
:104D6000880F991F3A95E1F7482B592B878199278E
:104D700080779070B4E095958795BA95E1F7482BC8
:104D8000592B283041F4BA01C8010E945410809177
:104D9000720382602BC080917203816080937203E2
:104DA000F601878180FD05C0809172038260809347
:104DB0007203F6016481858186FD6068C8010E94E6
:104DC0000C1016C0F6018581282F3327868199277C
:104DD0009695982F882797958795282B392BB90179
:104DE00084810E946E1080917203846080937203AC
:104DF0000E94D30E9CC1F6018281082F1127838166
:104E000099279695982F882797958795082B192B82
:104E10008581282F3327A901542F4427550F550F7B
:104E2000868199278F77907033E0880F991F3A9584
:104E3000E1F7482B592B8781992780779070B4E050
:104E400095958795BA95E1F7482B592B648126FDF6
:104E50006068C8010E94CD0F6AC1F501858D968DED
:104E6000892B41F0A8E09A2E858D8F778983858DD7
:104E7000968D07C09924D5018C918F7789838D9168
:104E80009C91880F892F881F990B91958F778A8322
:104E9000F501808D80FF02C0F0E19F2A0E944C2323
:104EA0007B018C01862F8F778B83E7E01695079522
:104EB000F794E794EA95D1F78E2D8F778C8377E07E
:104EC00016950795F794E7947A95D1F78E2D8F77FD
:104ED0008D8367E016950795F794E7946A95D1F767
:104EE0008E2D877089298E83AE014F5F5F4F6BE0F7
:104EF0008FEF0E9400261BC10E944C237B018C0176
:104F0000DC01CB018F779070A070B070F601248126
:104F100033274427552782179307A407B50709F0BD
:104F200030C1D801C70180789F73A070B07057E07E
:104F3000B695A795979587955A95D1F725813327EB
:104F40004427552782179307A407B50709F019C10D
:104F5000D801C7018070907CAF71B0704EE0B695FB
:104F6000A795979587954A95D1F7268133274427AA
:104F7000552782179307A407B50709F002C180E0FF
:104F800090E0A0EEB0E0E822F9220A231B2335E1ED
:104F900016950795F794E7943A95D1F72781822FD4
:104FA0009927AA27BB2787709070A070B070E81669
:104FB000F9060A071B0709F0E4C0922E969496940E
:104FC00096948281082F1127838199279695982F8F
:104FD000882797958795082B192B0115110509F43A
:104FE000D0C0E92CFF24E0FE09C0C5014F96AC01FA
:104FF00060E070E0C8010E94292A8C0101151105AA
:1050000029F0B801809143010E94CA23D5018D91F6
:105010009C91892B09F4B5C0E1FEB3C0F501808DE8
:105020008160808FAEC0F6018281282F3327838173
:1050300099279695982F882797958795282B392B10
:10504000309375032093740372C0F6018281282F78
:105050003327838199279695982F88279795879549
:10506000282B392B30937803209377038481809306
:105070008503858180937903868180937A0380916B
:10508000760381601CC0F6013296ABE7B3E094E092
:1050900081918D93915097FFFBCF80917603826031
:1050A0000EC0D6011296EBE7F3E093E08D91858375
:1050B0009150319697FFFACF809176038460809368
:1050C000760335C0F6018581882389F18281282FF6
:1050D0003327838199279695982F882797958795C9
:1050E000282B392B8481992790E4899F902D88273C
:1050F0001124282B392B20FF02C062E701C067E68C
:10510000C901969587950E94ED2C11C00E94362406
:10511000F60182810E94E6100AC0F601828188238E
:1051200021F00E942823FC0184810E94A50DD60154
:105130008C9199278F7790702091430133278217A4
:10514000930749F480917303882329F080917303B6
:10515000815080937303F501808D992796958795EB
:105160009C012170307080FD04C0A90160E0C9017C
:1051700006C0F50146815781628D808191810E9430
:10518000712426960FB6F894DEBF0FBECDBFDF9117
:10519000CF911F910F91FF90EF90DF90CF90BF9034
:1051A000AF909F900895FF920F931F93CF93F82E87
:1051B0008B014115510519F48FEF9FEF3FC0CA01D4
:1051C0000E946A259093DF018093DE011092E20134
:1051D0008EEF9FEF9093E1018093E001C091E20197
:1051E000FF2029F0A8016F2D80E00E94002684E0B6
:1051F0008093730306C080917303882331F00E946B
:10520000F8058091E2018823B1F30E94D124811135
:10521000C0E08091E201882319F4CF5FC83000F329
:105220008091DE019091DF010E946A251092DF01DA
:105230001092DE018091E0019091E101CF911F91E8
:105240000F91FF900895CF93DF93CDB7DEB72697E8
:105250000FB6F894DEBF0FBECDBF36E0FE0131962B
:1052600011923A95E9F74983AE014F5F5F4F0E9473
:10527000002626960FB6F894DEBF0FBECDBFDF9195
:10528000CF910895CF93DF93CDB7DEB726970FB6B2
:10529000F894DEBF0FBECDBF26E0FE01319611921D
:1052A0002A95E9F7282F2F772983880F892F881FC0
:1052B000990B91958F778A83AE014F5F5F4F63E1C2
:1052C0008FEF0E94002626960FB6F894DEBF0FBE21
:1052D000CDBFDF91CF9108959F92AF92BF92CF92B1
:1052E000DF92EF92FF920F931F93CF93DF93CDB78F
:1052F000DEB726970FB6F894DEBF0FBECDBFFC0118
:105300008B01942E6901672B11F0232B19F480E097
:1053100090E085C086E05E010894A11CB11CD50117
:105320001D928A95E9F754E1E52E8E2F8F778983B8
:10533000EE0FEF2FEE1FFF0BF1958E2F8F778A83E5
:1053400020E08E2D99278631910501F18731910555
:1053500034F48431910549F04597C9F024C0873170
:10536000910599F0489781F01EC0802F8F778B832D
:10537000C801880F892F881F990B91958F778C838F
:10538000892D8F778D830FC023E02D5F2D5F92E0F5
:10539000D5011296F601E20FF11D80818D93915097
:1053A0002F5F97FFF7CF1092750310927403FF24BD
:1053B0008091740390917503892B09F5AE014F5FBD
:1053C0005F4F6E2D8FEF0E94002685E08093730360
:1053D00006C080917303882341F00E94F8058091F4
:1053E000740390917503892BA1F3F3948091740356
:1053F00090917503892B19F489E08F15F8F6809147
:10540000740390917503009751F0E0917403F0914B
:105410007503E39488E18E1508F087CFCF012696B7
:105420000FB6F894DEBF0FBECDBFDF91CF911F91B5
:105430000F91FF90EF90DF90CF90BF90AF909F9033
:1054400008959A01462FBC0180E090E00E946C29EB
:105450000895DF92EF92FF920F931F93CF93DF9304
:10546000CDB7DEB726970FB6F894DEBF0FBECDBF1F
:105470009C017B018A0101978F5F934008F051C026
:1054800086E0FE01319611928A95E9F7822F8F7797
:105490008983220F232F221F330B3195822F8F7781
:1054A0008A8310927603DD2480917603873039F168
:1054B000AE014F5F5F4F60E18FEF0E9400268FE0EB
:1054C0008093730306C080917303882331F00E9498
:1054D000F805809176038730B1F7809176038730A5
:1054E00031F082B799278C599F4F0E94C20AD394FA
:1054F00080917603873019F089E08D15C8F6809188
:105500007603873021F4809179038F3769F4E114B1
:10551000F10411F0F70110820115110511F0F801E5
:10552000108280E090E018C0E114F10421F0809135
:105530008503F70180830115110551F08BE0F80117
:10554000A9E7B3E00D9001928A95E1F7F80113867F
:10555000809177039091780326960FB6F894DEBF7A
:105560000FBECDBFDF91CF911F910F91FF90EF90B4
:10557000DF9008950F931F93CF93DF93CDB7DEB7DE
:1055800026970FB6F894DEBF0FBECDBF062F26E0DC
:10559000FE01319611922A95E9F7282F2F7729835A
:1055A000880F892F881F990B91958F778A838FEFAA
:1055B0009FEF909375038093740310E080917403C0
:1055C0009091750397FF20C0AE014F5F5F4F602F32
:1055D0008FEF0E94002685E08093730306C08091C0
:1055E0007303882341F00E94F80580917403909121
:1055F00075039923A4F31F5F809174039091750341
:1056000097FF02C01A3000F38091740390917503E4
:1056100026960FB6F894DEBF0FBECDBFDF91CF91B7
:105620001F910F91089561E10E94BA2A089562E1E5
:105630000E94BA2A0895E82F109287038091870369
:1056400080938603809186038093A9038091A903A8
:105650008093A803119A1098199A189882E08BB930
:10566000E83008F0E1E0FF27EE0FFF1FEF5BF44F9B
:10567000A591B491653010F465E003C0693008F07D
:1056800068E04F7D6550660F453411F4606203C0D9
:105690004F3409F46063223008F068608B2F99273B
:1056A00087FD9A958F7080939000A9B960939500BB
:1056B00088EB8AB980E090E008951F920F920FB6B0
:1056C0000F9211248F939F93EF93FF939091A803D0
:1056D0008091A903981711F4559813C08091A903DC
:1056E000E82FFF27EA57FC4F84A18CB98091A903CA
:1056F0008F5F8093A9038091A903883010F01092E6
:10570000A903FF91EF919F918F910F900FBE0F9082
:105710001F9018951F920F920FB60F9211242F937E
:105720003F938F939F93EF93FF9380918603282F4E
:10573000332780918703992701972817390741F06C
:10574000809186038F3179F480918703882359F4FF
:10575000809187038F5F80938703809187038032D6
:1057600010F01092870380918603E82FFF27EA57F5
:10577000FC4F8CB18283809186038F5F8093860378
:1057800080918603803210F010928603FF91EF9192
:105790009F918F913F912F910F900FBE0F901F906F
:1057A000189550E060E070E027E0813D920708F036
:1057B00051E02FE0813A920708F052E023E289326B
:1057C000920708F053E026E3813B920708F054E08B
:1057D00026E48135920708F055E028E8893B9207D6
:1057E00008F056E0895D964D08F057E078948BB14B
:1057F000992726E0969587952A95E1F79C012170D7
:10580000307080FFB9016F5F7F4FA89587E26031EC
:10581000780768F321E04EE468E0852F0E941B2B97
:10582000089599278330910509F1843091054CF44E
:1058300081309105A9F082309105ACF4892B69F093
:1058400024C085309105C1F08530910594F08630F3
:105850009105A9F00797B1F018C080EB94E0089586
:1058600080E699E0089580EC92E1089580E895E261
:10587000089580E498E3089580E09BE4089580E033
:1058800096E9089580E091EE089580E090E0089513
:10589000089589B1282F3327809190009927982F58
:1058A0008827282B392B60E040E050E0FA01EF5BBD
:1058B000F44F859194918217930729F06F5F4E5FA3
:1058C0005F4F683098F3862F0E94112C0895482F5F
:1058D00006C08091A903882391F4559A7894A895DD
:1058E0008091A803282F33278091A9039927019736
:1058F0002817390791F38091A803873051F38091DD
:10590000A803E82FFF27EA57FC4F44A38091A80380
:105910008F5F8093A8038091A803883010F01092C5
:10592000A803559A80E090E00895909186038091B5
:105930008703981719F48FEF9FEF089580918703DD
:10594000E82FFF27EA57FC4F8281282F3327F8944E
:10595000809187038F5F80938703809187038032D4
:1059600010F0109287037894C90108950895CF929A
:10597000DF92EF92FF920F931F93CF93DF93E82E66
:10598000F62E8A016AEC0E94AA0D6F2D8E2D0E94C0
:10599000AA0DE80185E0C82ED12CC00ED11E0C1531
:1059A0001D0590F40881802F8A5C843028F46BEC0C
:1059B0008E2D0E94AA0D0F70602F8E2D0E94AA0DB1
:1059C0002196CC15DD0570F3DF91CF911F910F91DA
:1059D000FF90EF90DF90CF900895CF93DF93CDB7F6
:1059E000DEB726970FB6F894DEBF0FBECDBFDC0141
:1059F000262F86E0FE01319611928A95E9F7FE0185
:105A000031968B2F9927AF0189833196A1932F77F8
:105A1000208366E080E00E94B72C26960FB6F894AB
:105A2000DEBF0FBECDBFDF91CF910895FC01818114
:105A3000893121F0CF010E947C2508958481992726
:105A40000E94742508950895CF93DF93CDB7DEB7F4
:105A500026970FB6F894DEBF0FBECDBF96E0FE01CD
:105A6000319611929A95E9F78983AE014F5F5F4FA6
:105A700062E080E00E94B72C26960FB6F894DEBF55
:105A80000FBECDBFDF91CF910895CF93DF93CDB7F8
:105A9000DEB726970FB6F894DEBF0FBECDBF9C01D0
:105AA00086E0FE01319611928A95E9F7832F9927B6
:105AB00089832A83AE014F5F5F4F63E080E00E94DD
:105AC000B72C26960FB6F894DEBF0FBECDBFDF9180
:105AD000CF9108951092EE011092EF019091EE0196
:105AE0008A3C09F491E09093F0010895EF92FF92BF
:105AF0000F931F93CF93DF93CDB7DEB762970FB6A7
:105B0000F894DEBF0FBECDBF082F162F882309F0F3
:105B1000A6C164EEE62E61E0F62E8091EE018823A8
:105B2000A1F08091E4019091E501A091E601B0918E
:105B3000E7014496A11DB11DBC01CD010E94DE0804
:105B4000882319F0802F0E946A2D80914003909144
:105B50004103A0914203B09143038093E4019093E9
:105B6000E501A093E601B093E7011A3C11F4812FFF
:105B700074C18091F001882309F471C11B3C21F4A8
:105B800081E0F70183876BC18091EF018111106C77
:105B9000F70113868091EE01E82FFF27EC51FE4FAD
:105BA00014838F5FF7018287863008F458C10E9402
:105BB000C10E8C018091E80199278330910509F489
:105BC000B9C08430910554F48130910561F182307F
:105BD00091050CF053C0892B69F03AC185309105CD
:105BE00009F4CEC0853091050CF4B5C0069709F4D0
:105BF000F7C02EC16CEC80E00E94AA0DF801828DE6
:105C00008F8386819781892F9927888786818987C5
:105C10000E94F4058A871C861B86AE01495F5F4F90
:105C20006C85862F28C06CEC80E00E94AA0DF801DC
:105C300080819181892F99278F8380818887818DA9
:105C4000992783709070278D332727FD3095822BFD
:105C5000932B892B11F080E801C080E08987F8013F
:105C6000818D0E949C0E8A871C861B86AE01495F2F
:105C70005F4F61E08C850E94B72CEEC08091E901F6
:105C80009927F82EEE248091EA01E80EF11C80910C
:105C9000EC019927582F44278091ED01480F511DA1
:105CA000E114F10419F4F801E080F180F0E0EF165E
:105CB000F0E4FF0608F0CCC0F80180819181E8167D
:105CC000F90631F46091EB01C7010E94CD0F86C047
:105CD000FE0131968E2D8F779F0189833196EE0CD0
:105CE000EF2CEE1CFF08F1948E2D8F77819380911D
:105CF000EB018F778193CA01892F99278695869525
:105D0000982F9F7390838091EB0187FF02C090646E
:105D100090833196CA01A3E096958795AA95E1F7FD
:105D20008F778193842F8295807F8F778083A901DD
:105D300063E051C08091E9019927982F882720912D
:105D4000EA0160E0820F911D0E94260F882309F06E
:105D500045C06DEC7FC04091E901242F33272430EA
:105D6000310508F075C081E001C0880F2A95EAF777
:105D70008D7009F46DC060E280E00E9423292EC07E
:105D80008091E9019927F82EEE248091EA01E80E2E
:105D9000F11C86E0FE01319611928A95E9F7FE0129
:105DA00031968E2D8F779F0189833196EE0CEF2CE3
:105DB000EE1CFF08F1948E2D8F778193EE0CEF2C63
:105DC000EE1CFF08F1948E2D837081938091EB017E
:105DD0008083A90166E080E00E9400266CEC39C057
:105DE0008091E9019927F82EEE248091EA01E80ECE
:105DF000F11C86E0FE013D9611928A95E9F78E012D
:105E0000035F1F4FB701C8010E94642446E15DE2B1
:105E1000B80189E10E94D3288C018235910569F08F
:105E20008335910524F48734910539F011C0873604
:105E3000910519F08237910559F46CEC80E00E94CD
:105E4000AA0D802F8F77682FC7010E94ED2C04C008
:105E50006DEC80E00E94AA0D80E00E946A2D62969F
:105E60000FB6F894DEBF0FBECDBFDF91CF911F916B
:105E70000F91FF90EF900895E199FECF9FBB8EBBED
:105E8000E09A99278DB308954115510569F0DC0119
:105E9000E199FECF7FBB6EBBE09A6F5F7F4F0DB283
:105EA0000D9241505040B1F70895E199FECF9FBB4C
:105EB0008EBB6DBB0FB6F894E29AE19A0FBE0895BF
:105EC000DC0101C06D9341505040E0F70895FB01A3
:105ED000DC0101900D920020E1F708950F931F93CC
:105EE000CF93DF93CDB7DEB72C970FB6F894DEBF14
:105EF0000FBECDBF8C0136E03C8389839A832FEFA0
:105F00003FE72D833E83CE0101960E94C02FAF81D3
:105F1000B885A00FB11F1C922C960FB6F894DEBF67
:105F20000FBECDBFDF91CF911F910F9108950F93B9
:105F30001F93CF93DF93CDB7DEB72C970FB6F894AE
:105F4000DEBF0FBECDBF8C013EE03C8389839A83C8
:105F50002FEF3FE72D833E83CE0101960E94C02F95
:105F6000AF81B885A00FB11F1C922C960FB6F89484
:105F7000DEBF0FBECDBFDF91CF911F910F9108956E
:105F80002F923F924F925F926F927F928F929F9249
:105F9000AF92BF92CF92DF92EF92FF920F931F9337
:105FA000CF93DF93CDB7DEB762970FB6F894DEBF1D
:105FB0000FBECDBFAA24BB2465014C016D877E872F
:105FC0004F87588B44245524FC0146825782838195
:105FD00081FD5BC28FEF9FEF6FC240FE44C2862DF2
:105FE00080538A30E0F4F0E36F1641F42A892223CB
:105FF00029F4772019F480E091E08BC08AE09A8937
:10600000989F902D1124892F860D80538A8B882389
:1060100014F4EFE7EA8B43FC38C27A8836C243FEB9
:1060200005C0FA89FF2311F421E02A8B862D9927D8
:1060300087FD90958836910554F5853691050CF0CD
:106040006BC08835910509F4D3C089359105B4F446
:106050008B32910509F442C08C32910544F48032B0
:10606000910509F43FC0839709F442C0F2C18D3213
:106070009105D9F18E9709F440C0EBC183369105A3
:1060800009F454C08436910509F478C0E2C1803720
:10609000910509F4A5C08137910584F48C369105EA
:1060A000B1F18D3691052CF48936910509F466C05D
:1060B000D0C18F36910509F490C0CBC185379105C9
:1060C00009F498C08637910524F483379105B9F116
:1060D000C0C18837910509F48BC0BBC180E190E055
:1060E000482A592AE0E2F0E005C080E890E011C0BB
:1060F000E0E4F0E04E2A5F2AC8C188E090E0482A38
:10610000592AEFEFFEEF4E225F221A8ABEC184E0C9
:1061100090E0482A592AB9C10F2EFFE3AF2EF02D87
:106120007A940F2EF3E66F2EF02D3AC1EF85F889A1
:10613000CF0102968F87988BA0807A9431C1EF852A
:10614000F889CF0102968F87988BA080B18043FE9B
:106150000BC0EA898E2F992787FD9095BC01C50158
:106160000E94A832898B07C0F50101900020E9F751
:106170003197EA19E98BF9897F1A12C142FE0BC0E7
:10618000EF85F889CF0104968F87988B2081318124
:10619000428153810DC0EF85F889CF0102968F8728
:1061A000988B808191819C01442737FD4095542F25
:1061B00059016A01552364F4E2E0F0E04E2A5F2AB7
:1061C000D094C094B094A094A11CB11CC11CD11C4B
:1061D0008FEB9FEF482259222BC098E0998B0AC081
:1061E000E0E4F0E04E2A5F2A0F2EF8E76F2EF02D44
:1061F000F0E1F98B42FE0BC0EF85F889CF010496E0
:106200008F87988B20813181428153810BC0EF852C
:10621000F889CF0102968F87988B808191819C01AC
:106220004427552759016A01EFECFFEF4E225F2208
:106230001E010894211C311CF989EF2EFF24002730
:106240001127C601B501A80197010E94D332DC01D4
:10625000CB01F10180838A301CF0860D815203C08E
:10626000F1018081805DF10181931F01C601B501BB
:10627000A80197010E94D33259016A012115310505
:1062800041055105F1F6CE010196A22CA81AC201D2
:1062900082739070892B09F07A9446FE0FC0872D87
:1062A000992787FD9095F989F03131F40F2EFEEF93
:1062B0007F2EF02D780E02C0782E7A9443FE12C005
:1062C0008A89282F332727FD30958A2D9927821711
:1062D00093072CF0E7EFFFEF4E225F2203C0FA890D
:1062E000FA19FA8B43FE03C02A89721A01C07A1880
:1062F000C20180789170892B69F4872D7A941816E1
:106300004CF4B40180E290E00E947532872D7A94BB
:106310001816BCF341FE04C0B4018DE290E00BC03E
:1063200044FE04C0B4018BE290E005C045FE05C008
:10633000B40180E290E00E94753246FE0FC0B401C5
:1063400080E390E00E9475328989803139F4862D8E
:10635000992787FD9095B4010E94753250FE0DC0BB
:10636000872D7A9418164CF4B40180E390E00E94D3
:106370007532872D7A941816BCF343FE11C08A89B2
:10638000982F91509A8B18165CF4B40180E390E03A
:106390000E9475328A89E82FE150EA8B1816ACF317
:1063A000842D807869F4872D7A9418164CF4B40102
:1063B00080E290E00E947532872D7A941816BCF323
:1063C000F3E66F1641F48A2D992787FD9095B40165
:1063D0000E9475322DC023E76216B1F4898981507D
:1063E000898B8F3F29F1F5018081992787FD909551
:1063F0000894A11CB11CB4010E9475329989915076
:10640000998B9F3F81F714C0CE010196281639065B
:1064100079F08E010F5F1F4FF10182911F019927C3
:1064200087FD9095B4010E94753220163106A1F7C0
:10643000842D8078A9F0872D7A9418168CF4B401F5
:1064400080E290E00E947532872D7A941816BCF392
:1064500007C0862D992787FD9095B4010E9475325B
:106460004424552412C0F5E26F1641F44424552407
:1064700043941A8A7A882AE0298B07C0862D9927A7
:1064800087FD9095B4010E947532F401838183FFEA
:1064900008C0ED85FE85CF0101968D879E876490AB
:1064A00005C0ED85FE856190ED87FE87662009F0C9
:1064B00094CDF4018681978162960FB6F894DEBF81
:1064C0000FBECDBFDF91CF911F910F91FF90EF9045
:1064D000DF90CF90BF90AF909F908F907F906F9004
:1064E0005F904F903F902F9008950F931F93CF93FD
:1064F000DF938C01EB018B81992781FF22C082FF02
:1065000014C02E813F814C815D81241735073CF4F6
:10651000A881B9810D93A883B9832E813F812F5F14
:106520003F4F2E833F83C8010EC0E885F985802F39
:106530000995892B31F4EE81FF813196EE83FF833B
:10654000F2CF8FEF9FEFDF91CF911F910F910895C1
:10655000FC016150704001900110D8F78095909532
:106560008E0F9F1F0895991B79E004C0991F9617FD
:1065700008F0961B881F7A95C9F780950895AA1B85
:10658000BB1B51E107C0AA1FBB1FA617B70710F01E
:10659000A61BB70B881F991F5A95A9F78095909550
:1065A000BC01CD010895A1E21A2EAA1BBB1BFD015F
:1065B0000DC0AA1FBB1FEE1FFF1FA217B307E407E2
:1065C000F50720F0A21BB30BE40BF50B661F771F3A
:1065D000881F991F1A9469F760957095809590951A
:0A65E0009B01AC01BD01CF0108953D
:1065EA00FFFF00010000FF00007A1D080000AD1E39
:1065FA00FF00020000FF0000181DFF00006C18FFDA
:10660A000000B218FF0100081BFF0100C418FF01B7
:10661A0000311AFF01002A1CFF02007B1CFF020046
:06662A00C21CFFFF162652
:00000001FF
